:10000000A8050020552100005121000051210000C9
:1000100000000000000000000000000000000000E0
:10002000000000000000000000000000512100005E
:1000300000000000000000005121000051210000DC
:10004000512100005121000009030000512100004E
:100050000000000085060000000000000000000015
:10006000D5060000D10F00005121000051210000F1
:1000700051210000512100005121000051210000B8
:10008000000000000000000051210000512100008C
:100090005121000051210000512100005121000098
:1000A00051210000000000005121000051210000FA
:1000B00000000000512100005121000051210000EA
:1000C0000F4B104A984202D153695B0501E0536916
:1000D0005B045B0F09D1126803231340012B01D18C
:1000E00009480CE08020000209E0012B04D0022B1B
:1000F00004D1064B186802E0054800E00548704747
:100100000000014000020050001BB700000000206A
:100110001027000000805101F7B5061C0191171C43
:10012000FFF7CEFF0025041C430802209F4208D899
:10013000094A944201D91C1C0125201C391C02F0DB
:10014000A1F8019B011C2B430135336069437060AA
:10015000201C02F097F8FEBDFFFFFF00F0B585B050
:100160000393394B01911F68111C381C02F08AF867
:1001700005260290FF2501240298211C02F082F836
:1001800080235B04984213D8304A83181B0CDBB2DF
:100190001D1C022B00D20225EDB2291C02F072F8C0
:1001A00080235B02984203D8012808D086B207E07A
:1001B0006400013EE4B2002EDED1244E00E0061CB5
:1001C000211C6943381C714302F05CF8013D013E7B
:1001D000071CEDB2B6B2012C08D0022C08D0042CBA
:1001E00008D0083C631E9C41023404E0042402E071
:1001F000002400E001240198154B42081968D20040
:10020000FF209040814395400D431D60019A59683D
:1002100095000720A840221C0C1CAA4084431443CC
:100220005C6099680822AA400A439A60039B701C8C
:100230005843642102F026F8054A0138AD18686277
:10024000381CEE6005B0F0BD00000020FFFF00008C
:1002500000000440024BDA6D1143D9657047C04677
:1002600000000440F0B5174A85B00D1C6946041C17
:10027000C1CAC1C1126803200A60134A6B465169A2
:1002800000222263E060A260954218D08A01920F9A
:100290009200D65868083018291C01F0F3FF0B4B68
:1002A0000238984207D9E8003018291C01F0EAFF0B
:1002B0000009023802E0C0239B051843606205B0C4
:1002C000F0BDC046E423000000020050FFFF000024
:1002D000014B00225A607047FC000050054B5A68E1
:1002E000012A06D059225A6016225A6088225A6082
:1002F000F4E77047FC000050A023DB059A68012159
:100300000A439A6070470000C54BF0B504241C6294
:10031000C44B002219681A60012900D87FE1C24A43
:1003200002251068131C284200D1B6E01068C506EB
:1003300017D5BE4A01241078A0431070072903D8AE
:1003400011780919C9B21170B94811780078414083
:1003500011701278D10700D50BE11A6810218A4379
:100360005AE0106885067BD5106820420CD11368CE
:100370001C4314601068402398431060072900D97B
:100380004DE111680B4308E110688022904318602A
:10039000072902D819680A431A60196880201C6866
:1003A0000140402249082240914200D037E11A68BA
:1003B00004218A431A601C689D499E4A04422DD03C
:1003C00010780D789C4CC0B2EDB2255410780D78A1
:1003D0009A49C0B2EDB20D540020011C1578A84214
:1003E00004D8255C01306940C0B2F7E7002910D17C
:1003F000934A1160934A1170934A01211170934AF4
:10040000802110684900014311601A6890490A432D
:100410001A6019688F4A0A401A6000E110780028B3
:1004200005D108783F24A043802800D1A1E01078AE
:100430000D78814CC0B2EDB2255410780C787F490C
:10044000C0B2E4B20C5419682020814319601178BD
:100450000131C9B211701278102A00D989E0DEE0AA
:10046000734A10784000C0B21070072903D8117881
:100470000131C9B21170784A11780131C9B21170D5
:100480001178072905D91968202001431960002136
:1004900011701A6810210A43BEE7166880277F0290
:1004A0003E406D4863D08C1F012C04D811686B4B03
:1004B0000B401360AFE01268D4060FD5684A146889
:1004C00064081460082904D9146880218902214332
:1004D00011601A6810218A431A6012E0614A146898
:1004E00064081460082904D9146880218902214312
:1004F00011601A6810210A431A6002780132D2B2E0
:1005000002700278122A34D80278122A00D086E0CB
:10051000534A8020116880024908116051490C68D3
:10052000044202D1146820431060086814686040D7
:10053000106010684C4A904271D14C4A14680868A7
:10054000844211D13E4A00211160196801221143F1
:1005500019603D490A703D4A8021106849000143F5
:1005600011601968424A56E70968116001E00429E0
:1005700015D81A68950704D53E4A3F4912780120DC
:10058000885419683D4A0A401A60334A00231370A0
:10059000284A1370334A1360314A13603FE0082938
:1005A00039D9642908D913681A211F4317601368C1
:1005B0008B431360067032E00278122AD9D91A6888
:1005C000224206D01A6815431D601968234A0A4062
:1005D0001A601A6804210A431A601A6891071ED526
:1005E000244A254C1178632903D900211170217008
:1005F00004E00131C9B21170002262541A68082166
:100600000A431A6019681E4A0A401A60094A002300
:100610000370137003E003780133DBB20370F0BDA5
:10062000C040005038010020C4010020B00100206B
:10063000000100203C0100207C000020010100207E
:1006400078000020430100209F030020A003002029
:10065000010000100FFFFEFF9E030020FFFFFEFFC2
:10066000AC01002044010020FFFF03001401002022
:1006700001FFFEEF080000204801002000FFFEFF00
:10068000CBFFFEFF084B1A6A1A62084B1A6A1A62FD
:10069000074B1A6A1A62074A074B503219881278B8
:1006A0008A1892B21A80704780400050C0400050B3
:1006B00000410050910000208C0000204118884229
:1006C00004D00278024B01301A60F8E77047C04648
:1006D00000000540BB4B37B501229A60BA4B1A683F
:1006E00001321A60B94B1A6801321A60B84B1A7895
:1006F000632A03D81A780132D2B21A7018780138F6
:10070000102800D95CE101F0B3FD11001B005B0172
:1007100024005B0128005B015B016C0070005B0141
:100720005B015B015B015B015B01E900A94A527F50
:1007300010070CD5A84A1278002A00D040E106E044
:10074000A54A0F2112788A43702A00D038E164222A
:1007500049E0A24B0F221A7069E0A14A8021146877
:1007600049019C4B01A80C4219D014689D492140B5
:100770001160DA7C002A0ED15A7F910607D59C229F
:100780000270597C3F220A4097498A5C22E0A322EA
:100790000270AC221EE0A622027056221AE01468F3
:1007A00021431160DA7C002A0AD1597F3F228C064E
:1007B00001D59C7C00E05C788025AD00611903E0E8
:1007C0008024A40011193F242240874C8909615CD0
:1007D000A25C017042701B7F0221DD0700D4EFE0B4
:1007E000ECE0824B02221A70EAE0814B1A68900515
:1007F00035D580490A78D2B2501CC0B20870022A9E
:1008000003D919687C4A0A401A60724BDB7E59078B
:100810000FD5764B794902221A700B78724A9B09E0
:10082000D05C6E4B187008783F210140525C5A70C2
:10083000C6E01A0700D4C3E06C4B704903221A705B
:100840000B78694A9B09D318187F644B1870087895
:100850003F210140525C5A709A229A70B0E01968A8
:100860001022114200D1ABE065480178C9B24C1C9E
:10087000E4B20470022902D9196891431960614BEE
:100880001A881B88FF2A02D8DBB2002002E001335D
:10089000DBB201204F4AD17E0222CC070BD553494F
:1008A0000A7051499A09885C4C4A10703F200340F5
:1008B000CB5C537084E0114200D181E04B4A0321AC
:1008C000117049499A098A18147F444A14703F24C8
:1008D0002340CB5C53700B5C937071E03D4A137FF7
:1008E000111C9D076CD5537F980629D5464B547C27
:1008F0001878844264D15878927C824260D19A7888
:100900003648E42A02D09A78EC2A11D1344A126887
:10091000540106D5D9783D4A515C89090170DB78CC
:1009200024E0DA788A18527892090270DB7825E0A0
:100930009A78E72A02D09A78EF2A3CD1DB782FE028
:10094000254B5278187882423AD15A782348E42AC3
:1009500002D05A78EC2A1CD1214A1268550107D5D9
:1009600099782A4A515C890901709B78D25C07E02A
:100970009A788A185278920902709B78C9184A7836
:100980003F23134043700278174B9A5C0270427801
:100990000FE05A78E72A02D05A78EF2A0BD19B78D9
:1009A000772B08D1AC2303700D4B0F4A1B685B01FA
:1009B000DB0FD35C43700D4B1978C9B2FFF77EFE95
:1009C00037BDC0460000014038010020D0020020A1
:1009D00043010020910000207C0000203D01002008
:1009E000C4010020FFEFFFFFF42300001C010020E2
:1009F000A003002034010020FFFDFFFFA40300201E
:100A0000E50000208E00002001010020C801002028
:100A10000E4A802311681B010B4330B5136000237D
:100A20000B480C49C55CCC5CA54203D015680A4C48
:100A30002C4014600133102BF2D10023CA5CD2B2D7
:100A4000C2540133102BF9D130BDC046C40100207F
:100A50001D0100207C000020FFF7FFFF10B5144CA3
:100A6000FA22002192000123201CFFF777FB0121CD
:100A7000FA220B1C9200201CFFF770FB0221FA22C5
:100A80008A400123201CFFF769FBA2681223FF3371
:100A90001343A360074B00221A6019689C2292003E
:100AA0009142FAD9A268044B1340A36010BDC0461E
:100AB00000000440D0020020EEFEFFFFF0B5784BAE
:100AC00085B01A688023DB04051C0C1C134056D02B
:100AD000744E335C8B4200D1DFE0FFF7FFFB01F087
:100AE0009DFB7455704E802230689200AF088018CC
:100AF000BF00C01901F09AFB03231D409D40FF2356
:100B0000AB40021CAC409A431443011C2140351CED
:100B1000A14207D1306880239B00C018C01901F0A2
:100B200099FB27E0306880229200801801F060FB7A
:100B300000245E4B2868E318DE789A7836061204A3
:100B4000B6185A781B781202B618F61880239B0044
:100B5000C0180019311C01F07DFB2868802292002A
:100B600080180019311C01F075FB043480235B00F0
:100B70009C42DED101F024FBFFF7AAFB8DE001359A
:100B8000EDB20320532D00D988E0484E082D02D144
:100B90003370181C82E0735D8B4252D0FFF79EFBCE
:100BA00001F03CFB404FAB0038680193181801F08E
:100BB0003DFBC3B23A1CFF2B07D1984300190290AA
:100BC000019A3868029910180BE0FF2C10D02040D1
:100BD000A0420DD1631E3868019AFF3B10180293A2
:100BE000191C01F037FB3868019B0299181821E0A5
:100BF0001068745501F0FCFA00220192019A2A4F04
:100C0000B35C3868013BFF3B0293930018180299CC
:100C1000039301F01FFB3868039A0299101801F042
:100C200019FB019B01330193542BE7D1386820490C
:100C3000F930FF3001F00EFB01F0C2FAFFF748FB7C
:100C40007455312D0AD13136307864244121604306
:100C500001F066FB0021231A16480BE0322D0CD15F
:100C60003236307864244121604301F059FB231A65
:100C700010480121FA2292000DE0332D0DD13336B8
:100C8000307864244121604301F04AFB0221231A99
:100C9000FA2208488A40FFF761FA012005B0F0BD4A
:100CA000C4010020C8010020CC02002091000020D7
:100CB000785634120000044008B5FFF70FFB01F02E
:100CC000ADFA044B0021186801F0C4FAFFF714FBD9
:100CD00008BDC046CC020020074B1A68074B11061E
:100CE00003D59968064A0A4003E0996880225200B9
:100CF0000A439A60F0E7C046180100200000044053
:100D0000FFFEFFFFAA4AAB49F0B5156813680968F2
:100D1000A9488B43A94913600B7844789C4203D0BF
:100D2000002383700B78437014680023E60608D50F
:100D3000A34B1C68A34B670501D5023300E00333C6
:100D4000DB7F1468E60703D59E4C0434E47F23431D
:100D50001468A70703D59B4C0534E47F234314682C
:100D6000660721D5974CA61DF67F3343261C3536E2
:100D70003678F70605D50F780126374333430F70D1
:100D8000DBB2261C37363678F70604D50F780226F4
:100D900037430F70334336342478E60604D50E7893
:100DA000042426430E7023431468270721D5854C5D
:100DB000E61DF67F3343261C35363678B70605D553
:100DC0000F780126374333430F70DBB2261C3736CA
:100DD0003678B70604D50F78022637430F703343B1
:100DE00036342478A60604D50E78042426430E70E3
:100DF00023431168CF0503D572490831C97F0B43DE
:100E000011688C0503D56F49283109780B431168A7
:100E10004E0503D56B49293109780B4311680F053D
:100E200003D568492A3109780B431168CC0403D5EE
:100E300064492B3109780B4311688E0403D561494D
:100E40002C3109780B4311684F0403D55D492D31CE
:100E500009780B4311680C0403D55A492E310978DF
:100E60000B431168CE0303D55649403109780B4333
:100E700011688F0303D55349413109780B43116839
:100E80004C0303D54F49423109780B4311680E03D7
:100E900003D54C49433109780B431168CF0203D580
:100EA0004849443109780B4311688C0203D5454900
:100EB000453109780B4311684E0203D5414946314B
:100EC00009780B4311680F0203D53E494731097871
:100ED0000B431168CC0103D53A49483109780B43DB
:100EE00011688E0103D53749493109780B431168E0
:100EF0004F0103D533494A3109780B4311680C017E
:100F000003D530494B3109780B431168CE0003D526
:100F10002C494C3109780B4311688F0003D52949BE
:100F20004D3109780B4311684C0003D525494E31EA
:100F300009780B431268002A03DA224A4F321278EA
:100F4000134382789A422DD001211F4A0B4206D0CA
:100F50001A480078084202D09068014302E0916884
:100F600001208143916002210B4207D01348007891
:100F7000084203D091681020014302E091681020DC
:100F80008143916004210B4208D00C48007808424C
:100F900004D0906880214900014302E090680B4929
:100FA00001409160044A9370014B1D60F0BDC04642
:100FB00030010020FC00002008000020C8020020B2
:100FC000C40100209100002000000440FFFEFFFF4C
:100FD000CF4BF7B501229A60CE4BCF4C19688918D8
:100FE00019601968114200D1ACE0A388CB4A934242
:100FF00002D80133A3800AE0A2790023511CA17119
:10100000C749A38053310978914200D2A371208946
:101010000A21013080B2208101F078F98EB2002ED1
:1010200000D08FE0BF4DC04F2B789D20DBB20193E5
:101030003B8840005843642101F072F90199BB4A92
:101040004B0080B298522B780133DBB22B70297899
:101050002B1C151C642900D91E7000223A801B78B5
:101060006421DBB20133DBB2002064269E424041A2
:10107000404203405800285A0139C9B212180029C9
:10108000F0D1A74EE260331C52331B78002B01D005
:101090005A43E260E268E120331C513300011978C1
:1010A000504301F0EFF8A24901F0ECF8A14B051C08
:1010B0001A88E060824234D0A7790023BA00A218CF
:1010C0001061321C2381019753321278181C009250
:1010D0000099DAB28A4206D2974A99008F580133B2
:1010E000BC466044F4E7E06001F0CCF8914F80B278
:1010F0003880019F013FBF00E7193B69002B03D1F6
:10110000002D01D18B4F3D80331C50331B78002BB9
:1011100007D08A4B10211A680A431A60884B0022B4
:101120001A702289874B9A420CD9002323815036AA
:1011300032789A4206D0814A10201168014311602A
:101140007F4A1370764D804F6B7F804E580726D5AF
:101150007F4A1368591C1160EA7AC8214A439342B6
:101160001DD93B68102213433B607A4B1B68002B50
:1011700005D0236E784A934206D8013303E0236EEC
:10118000002B01D0013B2366216E8023DB003268F7
:10119000994201D9134301E0704B13403360336827
:1011A0009A0315D532686E4B500405D5594A11681B
:1011B0001122C80509D504E0564A116811224805D4
:1011C00003D5996891430A1C01E099680A439A6023
:1011D00050490B68DA0601D1FFF794FD231C6433F4
:1011E0001A78511C1970697A914210D800221A702D
:1011F000231C65331A7801321A70231C66331A785F
:1012000001321A70231C67331A7801321A70231CBA
:1012100065331B78002B04D1524A01201178814399
:1012200011702A1C3A32127800929A4204D14D4928
:101230000122087810430870291C3D310978009874
:1012400042189A4204DA474B01211A788A431A70ED
:10125000231C66331B78002B04D1424A02201178EC
:10126000814311702A1C3B32127800929A4204D1B9
:101270003C4902200A7802430A70291C3E31097851
:10128000009842189A4204DA364B02211A788A43AF
:101290001A70231C67331B78002B04D1314A0420B9
:1012A0001178814311702A1C3C32127800929A42C4
:1012B00004D12C4904200A7802430A70291C3F31CA
:1012C0000978009842189A4204DA264B04211A78C9
:1012D0008A431A703368590546D52B1C35331B7861
:1012E0009A0704D51F4B01211A788A431A702B1CC8
:1012F00036331B780222134203D01A4B19789143DC
:1013000019702B1C37331B7898074BD545E0C04626
:10131000200001401801002008000020E703000021
:1013200091000020900000208C000020D4020020BA
:1013300040420F008E00002018000020A003002073
:10134000E50000208713000030010020C4010020C8
:101350007800002070420050FF070000FFFBFFFFF5
:1013600000000440C80200202B1C35331B780122EA
:10137000134203D03D4B1978914319702B1C36331F
:101380001B78D90704D5394B02211A788A431A7081
:101390002B1C37331B78DA0704D5344B04211A7819
:1013A0008A431A703B6858071DD52B1C35331B78B0
:1013B000D90604D52D4B01211A780A431A702B1C2B
:1013C00036331B78DA0604D5284B02211A780A43F3
:1013D0001A702B1C37331B78D80604D5234B0421F5
:1013E0001A780A431A703B6819071CD52B1C353331
:1013F0001B789A0604D51D4B01211A780A431A70EE
:101400002B1C36331B789F0604D5184B02211A7803
:101410000A431A7037352B78980604D5134B0421EC
:101420001A780A431A70221C6832138801339BB25F
:101430001380FA22D200934217D900231A1C0C49B8
:10144000C95C002901D00132D2B20133642BF6D13C
:10145000084B80211A70084A890010680023014354
:101460001160064A683423801370F7BDC80200205B
:1014700048010020A4030020A00300203401002024
:10148000F0B585B0FEF72AFFD34ED44BD44AD549E8
:101490001A6031607321B160D349D44C0A600022D4
:1014A0008A609A6000F0BAFEC020800300F0BEFEA1
:1014B000051CCF4800F0BAFEA54211D000F090FE06
:1014C000C020800300F094FEC0208003211C00F0A7
:1014D000C1FEF021C648890100F0BCFE00F078FE94
:1014E00000F0B2FEC34E00253060306800F09EFE72
:1014F0003368A800C01800F099FEBF4C6055013554
:10150000542DF5D12378A52B04D1237DAA2B01D00E
:1015100004271EE0306800F06BFE2378002B04D116
:10152000B64B20211A680A431A600025237DAA2B96
:1015300003D0B34B4033EB5C6355615D3368A80067
:101540000139C018FF39013500F084FE542DEDD16A
:10155000DEE73068FD30FF30C01900F067FEA94DAE
:10156000010A7B191A1F1070DA1E11709A1E010CE5
:10157000013B000E11700437187082235B009F42FC
:10158000E7D13068F930FF3000F050FE9E498842C4
:101590000ED100F015FE237F202213421CD09B4960
:1015A00080200E68C004304393430860237713E023
:1015B0003068F930FF3000F04DFE01238F4A126889
:1015C0009006E6D45A1C1B0304D1914B01201968E4
:1015D00041401960131CF1E763782B70E379AB711C
:1015E000237AEB71637C2B74A37C6B74237FEB7683
:1015F000637F2B77231C3A331A78231C3D331978E9
:101600005118FF2901D9D2431A70231C3B331A7891
:10161000231C3E3319785118FF2901D9D2431A707F
:10162000231C3C331A78231C3F3319785118FF29A7
:1016300001D9D2431A70231C51331A78013A032A74
:1016400001D901221A70231C533319780F220A4042
:1016500001321A706F4A704B5F499A604B690426D9
:101660006E4D33434B61081C6D4A022100F098FD1A
:101670002E606C4E8021301C09056B4AFEF74CFD34
:1016800033688022D2051343336033688027BF0557
:101690003B433360654E80235B008021FA222B6040
:1016A000301C0905D200FEF737FD33688020C005E5
:1016B00003433360336880211F4380239B003760DE
:1016C0002B60C2239B00EA58594E090232400A435C
:1016D000EA50802240480521520200F061FD3E4957
:1016E00020234A69A0271A434A61524A28211160DF
:1016F0002B60C1239B00EA58FF051640C02212024E
:101700001643EE50E0235B01BB63231C3133187892
:1017100064264121704300F003FE474DFA22331A3C
:1017200092000021281CFEF719FD231C3233187883
:101730004121704300F0F4FDFA22331A9200012196
:10174000281C3334FEF70AFD20784121704300F055
:10175000E7FD0221FA22331A8A40281CFEF7FEFC1C
:10176000AB68364A281C1343AB600721FEF772FDB5
:101770003A6B334B334913403B633A6B0223FF33DD
:1017800013433B633048FEF76DFDFEF7A1FD2F4B81
:1017900007221A701D4B8022196892010A431A60B1
:1017A0001F1C1A4C2368DA07FBD523681D0700D5D8
:1017B00013E1274A274913682068DBB2CB18197D4B
:1017C0000D4B5E780096850446D5502947D1206898
:1017D000860349D4597047E0C04000500040005093
:1017E00055550000CFFF000080400050FEFF2FFF46
:1017F00004003000CC02002091000020A003002053
:10180000F4230000C801002078563412C4010020DF
:10181000504200500C0031000002005000E100E096
:101820000100010000000140A086010020000140ED
:10183000FF00FFFF8041005000000440440400000E
:10184000FEFEFFFE90D0030000000540C80200200D
:1018500014010020742400002068850304D4587FFC
:10186000860601D500F02BFCBA4C8020256880024A
:10187000054200D059705B788B4201D000F01FFC0C
:10188000236803420BD11468B34B1020E50502D541
:101890001C68204302E01C688443201C1860136805
:1018A0009B0ADAB2272A1CD0322A01D100F02CFC84
:1018B000362A06D0372A0CD0CD2A0CD0D82A0CD004
:1018C00001E03C230EE0DC2A09D0DD2A0AD1FF2307
:1018D00008E03F2306E0CF2304E0F02302E0FC23EE
:1018E00000E00F239B4A1068860324D41068840408
:1018F00021D40225202008242B4208D0234200D0E6
:10190000E4E3034217D014689448204012E02342D5
:1019100000D1EDE3034203D180201468C00004E04D
:1019200004208D4A1C0602D51468204302E0146886
:101930008443201C1060874E3268950403D43268BB
:10194000019C900344D501241C405A0701D5022272
:101950001443DD0602D504221443E4B27D4D58063B
:1019600003D508231C43E4B22EE0012C2CD1029BAA
:10197000019A0133DBB20293012A18D02B68980335
:1019800015D580232A68DB011A420CD00398744BCA
:10199000009A0138C0B25A70FFF790F82A68714B6C
:1019A00013402B6003E02A68039113432B60029DD0
:1019B000802D0DD9326880239B0213433360326837
:1019C000694B1340336003E02A68674B13402B6078
:1019D000634B009E01945E7071E32268634B644D1B
:1019E00013402360634B19782368C9B2D80500D42B
:1019F000D9E02B780F229343702B00D0D3E02368DB
:101A0000190500D48BE22A7803231340032B14D149
:101A10006B78772B11D1524BAA78197F2023002A9B
:101A200001D0194300E099432668534B22681B20DC
:101A300013402360FFF742F826602B789A0700D006
:101A40003DE36B784A4EDBB20093236858012AD5F8
:101A50002A780C2313400C2B25D1AB78002B0ED009
:101A6000AB78102B0BD0AB78112B08D0AB78122BA6
:101A700005D0AB781B2B02D0AB781C2B03D122688E
:101A80003D4B13402360B078F178C0B2C9B2FFF784
:101A900015F8002801D1FFF70FF922688023DB0435
:101AA0001343236009E0B078F178C0B2C9B2FFF700
:101AB00005F8002801D1FFF7FFF8009D542D00D94B
:101AC000FDE223688020C004184000D0F7E232789D
:101AD0000C231340082B05D00C2B58D0042B00D01E
:101AE000EDE24BE0B3781F229343E02B00D0E6E217
:101AF00001231F4907228C7814400A1CA04204DAF3
:101B00005B000130DBB2C0B2F3E78C781448E60624
:101B100010D589780C0704D55178401841781943BD
:101B200003E051784018417899435078C0B2FEF7ED
:101B3000C5FFDFE04A788978801842781340082290
:101B40000A4002D0002B00D0D4E0134300D0B6E20C
:101B5000D0E0C046C401002030010020FFFBFFFFA1
:101B600091000020FFBFFFFFFFDFFFFFFFFFFDFF32
:101B70007C0000203C010020FFFFFFFBB378AC4954
:101B800072788A1852789A4200D098E2B2E070785F
:101B9000B178C0B2C9B2FEF791FF002800D0A9E029
:101BA000FFF78AF8A6E02B782268002B04D1802367
:101BB0009B001343236035E09E4B134023609C4BF6
:101BC0005A7F96061DD52A78587C904212D16A78A1
:101BD000987C90420ED10223974A581ED45C013360
:101BE000E4B21454102BF7D1944B1A78013AD2B2C4
:101BF0001A7012E0DB7C002B00D160E28E4A127872
:101C000008E02A785878904207D0DB7C002B00D17E
:101C100055E22A789A4200D051E2874B5B78E42B58
:101C200000D14CE23A6880239B0413433B603A683E
:101C3000834B1F2013403B603A68824B824C134019
:101C40003B607D4B5A788243602A00D1B8E107D8C7
:101C5000202A52D0402A00D1B2E1002A0ED02EE232
:101C6000A02A00D1D9E103D8802A00D15AE126E286
:101C7000C02A00D109E2E02A5BD020E2032900D982
:101C80001DE25A78D00611D5597803220A40997876
:101C9000022A00D08039664BC9B2DA7C8A4200D170
:101CA0000DE21320D974FEF709FF08E25A780F23DA
:101CB0001340012B0AD0002B02D00F2B1AD0FEE1CB
:101CC0003A6880235B0013433B60F8E1584C637F24
:101CD0000E2B04D00E211D206177FEF7EFFEE37C72
:101CE000002B04D000211320E174FEF7E7FEFEF77D
:101CF00003FBE4E1FEF7B2FEE1E13A68910500D5AD
:101D0000DDE14B4AD27C002A02D019788A420BD1FD
:101D10009A78396852B2002A03DA8022D2000A4344
:101D200001E04A4A0A403A609B785A0600D1C6E16F
:101D30006FE13A68150500D4F1E05A78EC2A34D105
:101D40003A68560125D59A78002A12D19A78102A35
:101D50000FD19A78112A0CD19A78122A09D19A783F
:101D60001B2A06D19A781C2A03D12168384A0A40D6
:101D700022609878D978C0B2C9B2FEF79FFE0028D9
:101D800001D1FEF799FF22688023DB04134323600F
:101D900095E19878D978C0B2C9B2FEF78FFE0028D5
:101DA00000D08CE1FEF788FF89E15A78EF2A00D055
:101DB00085E19A78772A19D11D4ADD78117F202094
:101DC000234B002D05D0014380222068D20402431A
:101DD00003E00843107722681A40226025682268D1
:101DE0001B2013402360FEF769FE2560124A93789A
:101DF0001E2B00D863E193782A2B00D95FE19178FC
:101E0000144BD07859181F390870927801211F3A65
:101E100091400A1C10490888024392B20A800F4977
:101E20008A4200D04BE11A783E2A19D0FEF754FFBF
:101E300091000020FFFDFFFF7C0000203C010020FE
:101E4000FFFEFFFFFFDFFFFFC4010020FFFBFFFFDE
:101E5000FFFFFFFBB101002074000020FF0F000016
:101E60005A78012AE2D19A78002ADFD1DA78B22AA8
:101E7000DCD11A79012A14D15A79022A11D19A791E
:101E8000002A0ED1DA79002A0BD11A7A172A08D142
:101E90005A7A032A05D19A7A202A02D1DB7A152BA5
:101EA000C4D0FEF71BFA00F0B9F9994D0024286858
:101EB00000F09EF9974B28681E5DA700013EFF3E8B
:101EC0003818311C00F0C6F92868311C3818013464
:101ED00000F0C0F9402CEDD128688F49FD30FF306B
:101EE00000F0B8F900F07CF9C020800300F080F920
:101EF000C0208003894900F0ADF9F02188488901AC
:101F000000F0A8F900F064F9864B03211A680A432F
:101F10001A6000F055F9844A844B1A60FEE7FEF718
:101F200077FDCCE0042900D9C9E07A49804A4D7F89
:101F3000CC7CAE0729D51D78AC4211D1487D0F214C
:101F4000041C0C400E1CA6431568341C103C2C408D
:101F500014605C7813682040014019431160AEE0C2
:101F6000002C09D04C7D58780F21214088435870AF
:101F700010682039014001E01168814311606C4A0A
:101F8000116858781F23034097E01D780F20AC425A
:101F90000ED1497D15680C1C0440E443E4B2103CAA
:101FA0002C4014605C78136821400840184352E0CC
:101FB00011688143116011685B78184008434AE05A
:101FC00004297CD85348427F91070BD45D781021B7
:101FD000574A0D4202D01568294302E015688D4327
:101FE000291C11602268950569D4C27C002A02D0A0
:101FF00019788A420AD15A782168900603D580223E
:10200000D2000A4301E04B4A0A4022605B78D906BD
:1020100055D0494B00221A8051E004294FD85A78F4
:102020003C48D40622D51C78C57C414A4349A54288
:1020300013D1407D0F24061C2640F643F6B21568E6
:102040003602314329401160597800090C40136869
:1020500020400002C018106031E01068014011609B
:10206000116858780F2303401B020CE01A78C17CDA
:10207000914224D02E4A3249106801401160116803
:102080005B781B071B0C5B1818E022491A78C97C87
:10209000914214D05978264ADE2907D1106829497F
:1020A0000140116011689B781B0406E01168090269
:1020B000090A116011689B781B060B431360224BC1
:1020C000224A19680A401A60FFF76BFB184A8025FC
:1020D000034207D010682B4202D0044314602AE464
:1020E000A04327E4012014682B4200D120E41CE423
:1020F000034200D11FE40E4A10681E0602D50543B4
:10210000156018E4A84315E43023FFF7EBFBC04645
:10211000CC02002091000020A5AA55A57EFFAFFFAC
:102120000400300000C000500400FA050CED00E08F
:1021300030010020FFFBFFFF74000020FFF0FFFFD5
:10214000FF0FFFFFFFFF00FFC4010020FCFFFEFFA9
:10215000FEE7000008B500230C4A0D499A188A4290
:1021600004D20C49C95C01331170F5E70A4B0B4AE4
:10217000591C013B934203D200221A700B1CF6E754
:1021800000F01CF8FFF77CF908BDC04600000020F5
:1021900008000020A825000009000020A803002056
:1021A00010B5130E84698B40234312028361120A17
:1021B000C3698A40111C1943C16110BD70470000FA
:1021C000024B01211A688A431A60704700C0005010
:1021D000024B10211A688A431A60704700C00050F1
:1021E000024B10211A680A431A60704700C0005061
:1021F000094B2222DA60012258601A611869012114
:10220000054A0840FAD111684023194202D0012042
:10221000136040427047C04600C00050024B01218D
:102220001A680A431A60704700C00050054B00222C
:10223000DA60012258601A611A69D107FCD4014B97
:102240009868704700C00050014B58697047C046FD
:1022500000C00050054B2122DA60012258609960CD
:102260001A611A69D107FCD47047C04600C00050FB
:1022700003B47146490840004900095A49008E4498
:1022800003BC7047002934D00123002210B48842D7
:102290002CD301242407A14204D2814202D2090195
:1022A0001B01F8E7E400A14204D2814202D24900B6
:1022B0005B00F8E7884201D3401A1A434C08A04259
:1022C00002D3001B5C0822438C08A04202D3001BEF
:1022D0009C082243CC08A04202D3001BDC08224306
:1022E000002803D01B0901D00909E3E7101C10BC2A
:1022F0007047002801D00020C04307B4024802A163
:102300004018029003BDC046D90000000029F0D05B
:1023100003B5FFF7B9FF0EBC4243891A1847C04600
:10232000002941D010B4041C4C40A44601230022D3
:10233000002900D54942002800D5404288422CD3CC
:1023400001242407A14204D2814202D209011B01C7
:10235000F8E7E400A14204D2814202D249005B00C6
:10236000F8E7884201D3401A1A434C08A04202D32E
:10237000001B5C0822438C08A04202D3001B9C086F
:102380002243CC08A04202D3001BDC0822430028D1
:1023900003D01B0901D00909E3E7101C6446002C97
:1023A00000D5404210BC7047002806D003DB002057
:1023B000C043400801E08020000607B4024802A1A3
:1023C0004018029003BDC046190000000029EBD060
:1023D00003B5FFF7A7FF0EBC4243891A1847C04652
:1023E0007047C046001BB70000000000008051018C
:1023F00000805101ACAAA9A5A3A69C9A9995939691
:102400008E8D8BB1B2B4B874726C6A696563665CA8
:102410005A595553564E4D4B4771E8E4E2D1C9C560
:10242000D8D4D2CAC6CC78171B1D1E2E363A272BFD
:102430002D353933A503FFFFFFFFFF0C3E00FF0AD8
:10244000FFFFFFFFFFC0FF00FF00FFFFFFFFFF00D8
:10245000030EFFFFFF020401000000000000000067
:1024600000000000004040400000000000000000AC
:1024700000FFFFFF0000000000000000000000005F
:10248000000000000B0157045002510106085207DA
:1024900091B1BFA10305540412145513181A56190B
:1024A00092B257A215175816C1C959C5D9E15ADDBC
:1024B00093B35BA3CDD55CD1090B5D0A0F115E1000
:1024C00094B45FA40C0E600D363861373C3E623D1B
:1024D00095B563A5393B643A484A65494E00664F55
:1024E00096B667A64B4D684CC2CA69C6DAE26ADE88
:1024F00097B76BA7CED66CD23F416D4045476E462D
:1025000098B86FA842447043E5E771E6EBED72ECD2
:1025100099B973A9E8EA74E9F7F975F8FDFF76FE51
:102520009ABA77AAFAFC78FBC3CB79C7DBE37ADFE8
:102530009BBBC0ABCFD77CD3EEF07DEFF4F67EF53E
:102540009CBC7FACF1F380F21B1D811C21238222F5
:102550009DBD83AD1E20841F2D2F852E33358634DF
:102560009EBE87AE30328831C4CC89C8DCE48AE0B4
:102570009F538BAFD0D88CD424268D252A2C8E2B1C
:10258000A07B8FB0272990285F7369636865725FAD
:102590003E0100B2010200001703201500000000F8
:0825A0002F7369636865725F27
:0825A800008051011600000043
:00000001FF
